:10000000B201E3280408A70007128712871283169B
:10001000071287128712F030870583122708B2185B
:100020002F283A30A1009830A9203330A600442070
:100030001330A1008830A92044206430A820442037
:100040006430A8202230A600442028302E200C3016
:100050002E2006302E20B21427082F283214A60096
:10006000321C3D288712033C031C422842200730E3
:10007000A100D030A920031408003214FE3C03195B
:10008000DE288716A60E321C32100716F0308705C0
:1000900026080F3987040712A60E3218442832307A
:1000A000A82003140800B31329080319B317053057
:1000B000A8002730A300103069200330A300E830E7
:1000C0006920A30164306920A3010A306920240853
:1000D0007028A2002508A1002408A000BD20200847
:1000E000A000A8030319B313290803197A282802CA
:1000F000031808002008031DB313B31B0800303E8B
:10010000D9280F39A00083161F088F3910389F0097
:1001100083120310A00DA00D1F08C139200401385F
:100120009F000030A1003230A9209F149F1896280C
:10013000A1011E08DE28A301A200FF30A207031CB4
:10014000A307031CDE280330A100DF30A9209D286F
:10015000A101E83EA000A109FC30031CB228A007C1
:100160000318AF28A0076400A10FAF282018B828F3
:10017000A01CBC280000BC280800A501A401103068
:10018000A600210DA40DA50D2208A4022308031C1E
:10019000230FA5020318D3282208A4072308031855
:1001A000230FA5070310A00DA10DA60BC128200841
:1001B000DE28840031088A0030088200831303138C
:1001C0008312640008008316013091008312073007
:1001D0009900831699010B30850031308700831216
:1001E0009F13FE300320013003204C3003204D309C
:1001F00003203330032035300320203003205430D7
:100200000320453003204D3003205030032045307B
:100210000320523003204130032054300320553056
:100220000320523003204530032020300320FE30CD
:100230000320C030032052300320453003204130DA
:100240000320443003204530032052300320203067
:10025000032076300320313003204630032007305E
:10026000A300D0309C2000308120B800FE30032055
:100270000130032052300320453003204130032059
:1002800044300320203003204C3003204D30032025
:100290003330032035300320FE300320C0300320EC
:1002A00056300320613003206C300320753003206A
:1002B000653003203A30032020300320A90138089C
:1002C000A400A5010230B000B10153200130A30009
:0A02D000F4309C20332963006B29F1
:02400E00DC3F95
:00000001FF
